:10000C00FFFFFFFFFFFFFFFF0000FF0F4CA0B860DA
:10001C004C8D08000D2135499199361BCAD0FD60D5
:10002C00BE0407200C07A9008D00D3A9008D1AD09F
:10003C00AD1FD0F011BE0507200C07A9DF8D00D332
:10004C00A9088D1AD060A0804C6208A20886300ADC
:10005C0048A0009002A00220100768C630F008A249
:10006C000C200C074C3F0760A008AD1FD0F0D7AD9B
:10007C0000D330F6A9008D1AD0AAE8301EAD00D3FB
:10008C0010F8A9088D1AD0EC0A07B00B6649EC0BD6
:10009C0007263088D0D460244930CFA08C4C62081D
:1000AC00209B08A900A00485309848A004201007C4
:1000BC0068A8C630D0F388D0F0A432A9008532A24B
:1000CC0002200C079848B1324818653185316820F8
:1000DC003B0768A8C8F005C4004CCE07E633C4340F
:1000EC00D009A535C533D0064CE107EAEAEA4CB491
:1000FC0007A531A201200C07203B07A0014C620888
:10010C004C3607209B08A000A9FF8549A200AD1F13
:10011C00D0F0EDAD00D330F6A9008D1AD0E830EC5C
:10012C00AD00D310F8A9088D1AD0EC0A0790D7C8E7
:10013C00D0DAA432A9008532984820580768A8A5BF
:10014C0030AE0307D02691321865318531C8D00204
:10015C00E633C434D0E2A533C535D0DC205807A033
:10016C0001A530C531F002A08F4C6208D132F0D815
:10017C00A091AECC089AA9408D0ED4A9228D00D4A2
:10018C00A9388D02D3A9008D00D3A93C8D02D35878
:10019C006086348435A26C8632A20E8633AE030799
:1001AC00D006AAD0034C90074CF307A9388D02D384
:1001BC00A9608D00D3A93C8D02D3A9008D00D385F5
:1001CC0014A219E414D0FC8D0ED485318D00D4A961
:1001DC00088D1FD078BAE8E88ECC086000A90C8591
:1001EC000BA9C8850AA91A850F8DE802A96E850E80
:1001FC008DE702A9808D330AA244A90AA0264C8659
:10020C00E4A9F1A00D20300CA210A90C9D420320F2
:10021C00D3094CB90C18900138664820890CA203FC
:10022C00A9009DE002CA10FAA210A9039D4203A9DD
:10023C002B9D4403A90B9D4503A9049D4A03AD3393
:10024C000A9D4B0320D30920A30990B520A309B024
:10025C00FBA9079D4203A90A9D4503A9249D4403BC
:10026C00A9029D4803A9009D490320D309386E219A
:10027C000AAD220A9D4403AD230A9D450338AD24E3
:10028C000AED220A9D4803AD250AED230A9D490378
:10029C00FE4803D003FE490320D309ADE202D0058A
:1002AC00ADE302F00B201E0AA9008DE2028DE302E1
:1002BC004C3C09186E210AA210A9079D4203A90AF9
:1002CC009D4503A9229D4403A9029D4803A9009DB5
:1002DC00490320D309AD220A2D230AC9FFF00218C5
:1002EC006038602056E49830016048A90C9D4203A8
:1002FC002056E4682C210A3024C988D020ADE002B5
:10030C00D00CADE102D007A548300F4CC80CADE0C5
:10031C00028D220AADE1028D230A6C220A48A9083B
:10032C00A00E20300CA0006820570C4CB90C6CE2CD
:10033C000200C80C00005B0A440BCC0B790B1B0CA5
:10034C001D0C000086438444A001A9009143A9FF21
:10035C00C89143C8B124C99BF0089143C8C00DD0C3
:10036C00F360A9209143C8C00DD0F960A9008D039A
:10037C000785458546A52A290CC904F035C908F01E
:10038C000160A002B124C956F025A90420FCFD305F
:10039C001BA26BA00E20340AA900A278A00E20810B
:1003AC0008201F0C983005A9808545604C8F0B38B0
:1003BC006646186647A90320FCFD30F0A901A27817
:1003CC00A00E208108C080F0E39830F0A238A00B7A
:1003DC0020340AA200BD390BC92FF00DC92AF01622
:1003EC00C940F00ADD6C0ED0D3E8E00CD0E7201F3A
:1003FC000CA001844560A2028A48BD6C0E20B0F2AC
:10040C0068AAE8E00CD0F1A2008A48BD250B20B008
:10041C00F268AAE8E006D0F1A9FF8DFC0220FDF2FB
:10042C00295F09404820B0F2A99B20B0F268C9545A
:10043C00F0BC4CAC0A2028542F4E2908A0D02086A2
:10044C00E4A24EA90BA0552086E4A24DA90BA0490D
:10045C002086E46CFEA446100A20CD0B98103EC0FA
:10046C0088D026A001A5451020A900A89143E643F9
:10047C00D002E644A91AC544D0EFA96EC543D0E911
:10048C00A900A26EA01A20810860A44610188D3213
:10049C000A20CD0BC000300DCD320AF008A091A976
:1004AC00008546854560A4453003A08760A0009177
:1004BC0043E643D002E644EE6C0ED003EE6D0EAD77
:1004CC006D0EC90CF003A00160A900A26EA01A2049
:1004DC008108981004A9008545201F0C60A445884C
:1004EC00F003A08360AD6C0E0D6D0ED022A54710ED
:1004FC0003A08860A901A26EA01A20810820270CF5
:10050C0098309CA90CCD6D0EF005386647D0D6A05E
:10051C0000B14348E643D002E64438AD6C0EE90125
:10052C008D6C0EAD6D0EE9008D6D0E68A00160A98D
:10053C00008D6C0E8D6D0EA90E8544A96E854360E1
:10054C00A20084CC85CB1869029D44039869009D58
:10055C004503A000B1CB9D4803C8B1CB9D4903A96D
:10056C000B9D42034C56E485D484D520AAD920E6B1
:10057C00D8A90085CDF00520B0F2E6CDA4CDB98088
:10058C000510F4498020B0F24C820CA92020B0F266
:10059C00E6CDA906C5CDD0F360A93E20B0F2A200ED
:1005AC00A9059D4203A90B9D4503A92B9D4403A9B5
:1005BC000E9D4803A9009D49032056E41004C089F0
:1005CC00D016BC480388F01060A913A00E20300C84
:1005DC00A9FF8DFC0220FDF2A2FF9AA9018509A9B1
:1005EC0000852BA90C852A208EEFA925A00D203083
:1005FC000CAD330A100AA9E8A00D20300C4CF70CF6
:10060C00A9E0A00D20300CA958A00D20300CA9FF9A
:10061C008DFC0220FDF2295F4820B0F268A006D9BB
:10062C00210EF0058810F830AF980AA8B9290E48A9
:10063C00B9280E48603100CBE1F3E5F4EFF7F9A0EF
:10064C00F3F9F3F4E5EDA0EFF0E5F2E1E3F9EAEE0E
:10065C00F9A0D7DAE1E2A0B2D4B1B29B9B7F2050D3
:10066C00727A657277793A2086009B9B7F7FA0CD4A
:10067C00A0C5A0CEA0D5A09B9BCC2D4C61646F7760
:10068C00616E696520706C696B7520D22D4C61644C
:10069C006F77616E696520692073746172749BD386
:1006AC002D53746172742070726F6772616D752056
:1006BC00201B9D2D5A696D6E792073746172749B29
:1006CC00C52D537465722E2073696C6E696B6965E8
:1006DC006D20D02D50727A657277799BC32D506F37
:1006EC0077726F7420646F204241534943419B9B46
:1006FC000600444C5547494507004B524F544B4953
:10070C004515009B7FFD5A6C7920666F726D617484
:10071C0020706C696B75202109009B7F7FFD426CFA
:10072C0061643A0C009B7F7FDBD2C5D4D5D2CE5D01
:10073C001E4C525350451D4304090709090A350E36
:10074C00400E630E500EAD330A49808D330A4CC8EF
:10075C000CAD02D349088D02D3A9038D0FD24CC81E
:10076C000CADF803D0F8A9FD8D01D320610E6CFA05
:10077C00BF6CFEBFA9018D44026CFCFFA9CD8502A4
:10078C00850CA9088503850D20CD08A966A00F202E
:10079C00300CA9FF8DFC0220FDF2295F0940482096
:1007AC00B0F2A99B20B0F268C94BD0034CC80FC95A
:1007BC0042F018A90E850BA9AC850A60A90C850B13
:1007CC00A9C8850AA90085084CC80CA9C4850AA922
:1007DC000E850B60A9A0856AA900852BA90C852A1A
:1007EC00208EEFA9C8850AA90C850BA9008508A93C
:1007FC00008DF803A9FD8D01D320EF0E6CFABF6CB0
:10080C00FEBFA9008D2F028D00D4A989A00F203026
:10081C000CA9008D0ED478A9228D2F028D00D4A99D
:10082C00008DFA03A2FFA0FFAD13D0CDFA03D0F4D4
:10083C0088D0F5CAD0F0A9408D0ED45820CD08A987
:10084C000E8503850DA96C8502850CA9008D4402CB
:10085C00A9018509A9FF8DF8038D01D3A91A853546
:10086C00A06EA9008534A2C09134C8D0FBE635E453
:10087C0035D0F56CFCFF2100CE2D4B534F2020C200
:10088C002D4B534F2642415349432020CB2D4B4FE8
:10089C0050494F57414E49C51E1100437A656B6153
:1008AC006A2E2E2E2E2E2E2E2E2E2E9BA90085320B
:1008BC00A9078533A9048534A9B08535A000B134C6
:1008CC009132E632D002E633E634D002E635A9C0E6
:1008DC00C535D0EA4CF20E60ADE90F8D8004EEC93F
:1008EC000FD003EECA0FEECC0FD003EECD0FA9172D
:1008FC00CDCA0FD0E34C8004004C360B0D2135498A
:10090C009199361BCAD0FD60BE8304208B04A900CC
:10091C008D00D3A9008D1AD0AD1FD0F011BE840468
:10092C00208B04A9DF8D00D3A9088D1AD060A0807C
:10093C004CD305A20886300A48A0009002A00220E1
:10094C008F0468C630F008A20C208B044CBE0460E7
:10095C00A008AD1FD0F0D7AD00D330F6A9008D1A8A
:10096C00D0AAE8301EAD00D310F8A9088D1AD0EC2F
:10097C008904B00B6688EC8A04263088D0D46024B5
:10098C008830CFA08C4CD305200606A900A0048586
:10099C00309848A004208F0468A8C630D0F388D0C3
:1009AC00F0A432A9008532A202208B049848B132FF
:1009BC004818653185316820BA0468A8C8F005C4A8
:1009CC00004C4D05E633C434D009A535C533D006EB
:1009DC004C6005EAEAEA4C3305A531A201208B04F0
:1009EC0020BA04A0014CD3054CB504200606A00087
:1009FC00A9FF8588A200AD1FD0F0EDAD00D330F675
:100A0C00A9008D1AD0E830ECAD00D310F8A9088DF0
:100A1C001AD0EC890490D7C8D0DAA432A900853258
:100A2C00984820D70468A8A53091321865318531D3
:100A3C00C8D002E633C434D0E7A533C535D0E120A5
:100A4C00D704A001A530C531F002A08FA68E9AA9BB
:100A5C00408D0ED4A9228D00D4A9388D02D3A900C3
:100A6C008D00D3A93C8D02D3586086348435A236D0
:100A7C008632A20B8633AAD0034C0F054C7205A903
:100A8C00388D02D3A9608D00D3A93C8D02D3A90067
:100A9C008D00D38514A219E414D0FC8D0ED48531AD
:100AAC008D00D4A9088D1FD078BAE8E8868E6041F5
:100ABC00062907AF075E07FE070008A900858F858A
:100ACC00838582A52A290CC904F035C908F0016078
:100ADC00A002B124C956F025A90420FCFD301BA2AC
:100AEC0035A00B205208A900A242A00B20F1052032
:100AFC000208983005A9808583604C72073866829D
:100B0C00186681A90320FCFD30F0A901A242A00BBC
:100B1C0020F105C080F0E39830F0A21DA007205210
:100B2C0008A200BD1E07C92FF00DC92AF016C94036
:100B3C00F00ADD360BD0D3E8E00CD0E7200208A099
:100B4C0001848360A2028A48BD360B20B0F268AAE9
:100B5C00E8E00CD0F1A2008A48BD0A0720B0F26888
:100B6C00AAE8E006D0F1A9FF8DFC0220FDF2295F76
:100B7C0009404820B0F2A99B20B0F268C954F0BCDF
:100B8C004C91062028542F4E2930313233343536CF
:100B9C0037383941424344303132333435363739C2
:100BAC00304142A482100A20B00798103CC088D073
:100BBC0026A001A5831020A900A89184E684D00268
:100BCC00E685A917C585D0EFA938C584D0E9A90059
:100BDC00A238A01720F10560A4821016859020B0D1
:100BEC0007C000300CC590F008A091A90085828543
:100BFC008360A4833003A08760A0009184E684D036
:100C0C0002E685EE360BD003EE370BAD370BC90C75
:100C1C00F003A00160A900A238A01720F1059810DC
:100C2C0004A900858320020860A48388F003A083B4
:100C3C0060AD360B0D370BD022A5811003A0886058
:100C4C00A901A238A01720F105200A0898309CA908
:100C5C000CCD370BF005386681D0D6A000B1844896
:100C6C00E684D002E68538AD360BE9018D360BAD46
:100C7C00370BE9008D370B68A00160A9008D360B8E
:100C8C008D370BA90B8585A938858460A20084CC8F
:100C9C0085CB1869029D44039869009D4503A0000B
:100CAC00B1CB9D4803C8B1CB9D4903A90B9D420311
:100CBC004C56E4484A4A4A4A20450868290FC90A52
:100CCC00B0040930D00269364CB0F286848485A019
:100CDC0001A9009184A9FFC89184C8B124C99BF0D3
:100CEC00089184C8C00DD0F360A9209184C8C00DB0
:100CFC00D0F960303132333435363738393031321F
:100D0C0033343536373839308589A200A9059D42F0
:100D1C0003A9089D4503A97A9D4403A9139D480383
:100D2C00A9009D49032056E41004C089D02020D886
:100D3C0008A9039D4203A9089D4503A97A9D440374
:100D4C00A5899D4A03A58D9D4B032056E4604C114B
:100D5C000AA210A90C9D42034C56E407009BFD42CD
:100D6C006C61643AA00BD002A0078C5203A0008CDB
:100D7C0058038C5903A2102056E460984820D808D8
:100D8C00A9E2A00820130868203A0820630A4C0244
:100D9C000AA58B8586A58C85874C2F09A91C858770
:100DAC00858CA9008586858BA904208F0830CC20E2
:100DBC00EF08301848208D09B02A20750986CB849D
:100DCC00CCA0006891CB2081094C3609A586858B77
:100DDC00A587858CC088F0034C020920D8082063B5
:100DEC000A4C020AA919A00B2013084C020A78A974
:100DFC00008D0ED4A9FE8D01D360A9FF8D01D3A95E
:100E0C00408D0ED45860A487A686E8D001C886868B
:100E1C008487C0F8B00AC0D0900598186908A81843
:100E2C0060A91C8587A9008586A908208F08100356
:100E3C004C0209208D09A58CC5879020D006A58B66
:100E4C00C586901820750986CB84CCA000B1CB4800
:100E5C002081096820EB0810DA4C020920D80830F0
:100E6C00F820630A4C020AA58D4980858D4C110A25
:100E7C00AD02D349088D02D34C110AA987A00A20D0
:100E8C001308A9FF8DFC0220FDF2A995A00A2013DE
:100E9C0008A9038D0FD2A58D3007A9D4A00A4C2C1C
:100EAC000AA9CAA00A201308A9DEA00A201308A9BF
:100EBC00FF8DFC0220FDF2295F4820B0F2A93E20F4
:100ECC00B0F268A004D9780AF0068810F84C110A20
:100EDC00980AA8B97E0A48B97D0A4860A92AA00BCD
:100EEC00201308A58C38E91C203A08A58B203A0859
:100EFC0060494F5350412209A709F609ED0917091A
:100F0C000C009B7F7FDBD2C5D4D5D2CE5D1E3300C7
:100F1C007D545552424F20434F505920322E31327E
:100F2C002028632920575A61622050494153544F5D
:100F3C005720313938389B9B7F7F50727A65727796
:100F4C00793A2008004B524F544B49452008004435
:100F5C004C55474945202039009B9B492D57637AB6
:100F6C007974616E696520412D446F6C61637A659B
:100F7C006E6965204F2D5A617069739B502D5072AC
:100F8C007A65727779202020532D53696C6E696BCA
:100F9C009B9B0F009B5A6120646C75676920706C79
:100FAC00696B9B0A009B446C75676F7363203AA94D
:100FBC0017850F8DE802A938850E8DE702A91C85CF
:100FCC006AA9FF8D4402A900852BA90C852A208EC5
:100FDC00EFA980858DA244A906A0362086E4900A4C
:100FEC00A9069D1B03A9369D1A034C110A0000008B
:100FFC0000000000000000000000000000000000E5
:10100C0000000000000000B0000403B0FFFFFFFF71
:10101C00FFFFFFFFFFFFFFFFFFFFFFFFFFFFFFFFD4
:10102C00FFFFFFFFFFFFFFFFFFFFFFFFFFFFFFFFC4
:10103C00FFFFFFFFFFFFFFFFFFFFFFFFFFFFFFFFB4
:10104C00FFFFFFFFFFFFFFFFFFFFFFFFFFFFFFFFA4
:00000001FF
